:020000040000FA
:04080000F3EF25F0FD
:0408080005EF25F0E3
:04081800C2EF24F017
:06082A0000C0E5FF01C063
:10083000E5FF02C0E5FF03C0E5FF04C0E5FF05C01A
:10084000E5FF06C0E5FF07C0E5FF08C0E5FF09C0FA
:10085000E5FF0AC0E5FF0BC0E5FF0CC0E5FF07019F
:100860006E51D8B4C1EF08F00701799779956FC739
:1008700000F0010E016E60C002F00250230A02E097
:1008800019EF07F0020E005CD8A0C1EF08F061C0BC
:1008900002F00250530A01E089D00050040A02E03D
:1008A000C1EF08F0030E016E62C002F00250036E49
:1008B000D00E0324026E0A0E025C05E30250036EA2
:1008C000F90E0324026E600E0124036E046A000E0A
:1008D000042203C0E9FF04C0EAFFEFCF03F0035096
:1008E000046ED00E0424036E0A0E035C05E303506D
:1008F000046EF90E0424036E100E025CD8B0C1EF32
:1009000008F0100E035CD8B0C1EF08F00238F00B0D
:10091000046E035004260450D8B4C1EF08F0800ED2
:10092000045CD8B0C1EF08F00438E8441F0B056E32
:10093000F00E0524066E076A020E072206C0E9FFC4
:1009400007C0EAFFEFCF08F0070E0414096E010E8E
:100950000A6E095005E0E86CD8900A36010FFDE3F5
:100960000A50081206C0E9FF07C0EAFF08C0EFFFFF
:10097000066A240E0526070E062205C0E9FF06C0FA
:10098000EAFFEFCF07F00A1E0A50071605C0E9FF7D
:1009900006C0EAFF07C0EFFF04500701765DD8B03C
:1009A000C1EF08F004C076F7C1EF08F00250430A27
:1009B00001E080D00050040A02E0C1EF08F0030E0D
:1009C000016E62C002F00250056ED00E0524026E68
:1009D0000A0E025C05E30250056EF90E0524026E54
:1009E000600E0124056E066A000E062205C0E9FFAE
:1009F00006C0EAFFEFCF03F00350056ED00E0524CA
:100A0000036E0A0E035C05E30350056EF90E052420
:100A1000036E100E025CD8B0C1EF08F0100E035C3C
:100A2000D8B0C1EF08F00238F00B0324046E045074
:100A3000D8B4C1EF08F0800E045CD8B0C1EF08F064
:100A40000438E8441F0B056E240E0524066E076A61
:100A5000070E072206C0E9FF07C0EAFFEFCF08F044
:100A6000070E0414096E010E0A6E095005E0E86CC9
:100A7000D8900A36010FFDE30A1C096E081606C05D
:100A8000E9FF07C0EAFF08C0EFFF066AF00E05267F
:100A9000020E062205C0E9FF06C0EAFFEFCF07F00D
:100AA0000750091605C0E9FF06C0EAFF09C0EFFFBD
:100AB000C1EF08F00250690A0EE1000EE56E390E32
:100AC000E56E800EE56E1FEC23F0030EE12695EC3B
:100AD00021F0C1EF08F002504C0A01E092D0000E64
:100AE000E56E390EE56E920EE56E1FEC23F0030EF7
:100AF000E12670C707F0070EE56E790EE56EE56A30
:100B00000750E56E000EE56E390EE56EA40EE56E3B
:100B10001FEC23F0070EE126056A010E066E065053
:100B20000701765DD8A066D00638E8441F0B076E33
:100B3000F00E0724086E096A020E092208C0E9FFB8
:100B400009C0EAFFEFCF08F0070E0614096E010E88
:100B50000A6E0B6A095006E0E86CD8900A360B362C
:100B6000010FFCE30C6A0A5008160B500C160850D3
:100B70000C10D8B43DD0086A240E0726070E0822B0
:100B800007C0E9FF08C0EAFFEFCF07F0086A075087
:100B90000A1608500B160A5005E10B5003E10A6AC9
:100BA0000A2A01D00A6A0A50D880E866D8900A6AF0
:100BB0000A36076A0ABE076806C008F00750E56EE5
:100BC0000A50E56EE56A0850E56E000EE56E390ED6
:100BD000E56ECA0EE56E1FEC23F0070EE126052A2E
:100BE00005500F0B05E10A0EE56E97EC26F0E65274
:100BF000062A95D70A0EE56E97EC26F0E652C1EF6D
:100C000008F00250460A13E1070179990701706B59
:100C10008B809D9A9D98000EE56E390EE56ED20E82
:100C2000E56E1FEC23F0030EE126C1EF08F0025041
:100C3000560A0CE1000EE56E390EE56EEA0EE56E21
:100C40001FEC23F0030EE126C1EF08F00250520A18
:100C500001E044D0000EE56A89EC26F0046EE6520D
:100C60000F0E0414056E0A0E055C08E205C006F0BE
:100C7000076A300E0626D8B0072A07D0086A055042
:100C8000370F066E000E0820076E04380F0B056E36
:100C90000A0E055C08E205C008F0096A300E082655
:100CA000D8B0092A07D00A6A0550370F086E000E1F
:100CB0000A20096E0750E56E0650E56E0950E56E94
:100CC0000850E56E000EE56E3A0EE56E1C0EE56E00
:100CD0001FEC23F0070EE126C1EF08F00250570A7F
:100CE00001E040D0030E016E62C002F00250056EBA
:100CF000D00E0524026E0A0E025C05E30250056E5A
:100D0000F90E0524026E600E0124056E066A000EBF
:100D1000062205C0E9FF06C0EAFFEFCF03F003504B
:100D2000056ED00E0524036E0A0E035C05E3035026
:100D3000056EF90E0524036E100E025CD8B0C1EFEB
:100D400008F0100E035CD8B0C1EF08F00238F00BC9
:100D50000324E56E000EE56A69EC1CF0E652E652EB
:100D6000C1EF08F00250450A21E1020E056E0701AD
:100D70006F51055C14E205C006F0052A076A600E93
:100D80000626000E072206C0E9FF07C0EAFFEFCFE4
:100D900002F00250E56E97EC26F0E652E8D70A0E14
:100DA000E56E97EC26F0E652C1EF08F00250440AD7
:100DB00002E0C1EF08F00050040A02E0C1EF08F0C1
:100DC000030E016E62C002F00250056ED00E0524C3
:100DD000026E0A0E025C05E30250056EF90E052450
:100DE000026E600E0124056E066A000E062205C022
:100DF000E9FF06C0EAFFEFCF03F00350056ED00E07
:100E00000524036E0A0E035C05E30350056EF90E1C
:100E10000524036E100E025CD8B0B3D1100E035C33
:100E2000D8B0AFD10238F00B0324046E04C074F7BD
:100E3000A8D10250210A01E03DD00006010E005C5D
:100E4000D8A09FD1010E07017B6F0001A06B0701A5
:100E50007C6B61C002F00250420A0FE00250490A66
:100E60000CE002504E0A09E00250520A06E002501D
:100E7000500A03E00250460A15E107017985025045
:100E8000460A0DE107017989000EE56E3A0EE56E1E
:100E9000260EE56E1FEC23F0030EE126AAD0070113
:100EA0007999A7D00250620A01E06BD1020E016E5F
:100EB00000069FD0070179A957D00028056E0001D0
:100EC000A06F05C07CF70250A16F07017C27020EBE
:100ED00007017B6F010E056E07016F51055C21E272
:100EE000A00E07017B25066E076A000E072205C0CB
:100EF00008F0052A096A600E0826000E092208C0BB
:100F0000E9FF09C0EAFFEFCF08F006C0E9FF07C01C
:100F1000EAFF08C0EFFF085007017C2707017B2B81
:100F2000DBD7A00E07017B25056E066A000E0622A0
:100F300007017C51076E076C05C0E9FF06C0EAFF98
:100F400007C0EFFF07017B2907017D6F07017E6B5B
:100F50008B909D9AA0C0ADFF010E07017B6F040E20
:100F60000701706F9D880DD1030E005CD8A009D1D8
:100F70000250056ED00E0524026E0A0E025C05E3D7
:100F80000250056EF90E0524026E020E016E61C05C
:100F900003F00350056ED00E0524036E0A0E035CA9
:100FA00005E30350056EF90E0524036E100E025C76
:100FB000D8B0E7D0100E035CD8B0E3D00238F00B05
:100FC0000324046E04AE03D00701798502D0070123
:100FD0007995049E0450D8B4D4D0010E07017B6FDC
:100FE00004500001A06F04C07CF7FE0E002607012C
:100FF0007987070179A502D0008E02D0D8900032FF
:10100000A00E07017B25046E056A000E052204C0B0
:10101000E9FF05C0EAFF00C0EFFF005007017C2791
:1010200007017B2B070179A528D001C000F007013B
:101030006F51005CD8B07FD0A00E07017B25046EF5
:10104000056A000E052200C006F0002A076A600E3D
:101050000626000E072206C0E9FF07C0EAFFEFCF11
:1010600006F004C0E9FF05C0EAFF06C0EFFF065026
:1010700007017C2707017B2BDAD707016F51015C41
:10108000D8B059D001C000F0012A046A600E0026D1
:10109000000E042200C0E9FF04C0EAFFEFCF02F017
:1010A0000250006ED00E0024026E0A0E025C05E3B0
:1010B0000250006EF90E0024026E07016F51015CB0
:1010C000D8B05FD001C000F0012A046A600E00268B
:1010D000000E042200C0E9FF04C0EAFFEFCF03F0D6
:1010E0000350006ED00E0024036E0A0E035C05E36D
:1010F0000350006EF90E0024036E100E025CD8B08F
:1011000040D0100E035CD8B03CD00238F00B032660
:10111000A00E07017B25006E026A000E022200C0AD
:10112000E9FF02C0EAFF03C0EFFF035007017C277D
:1011300007017B2BA2D7A00E07017B25006E016A59
:10114000000E012207017C51026E026C00C0E9FF13
:1011500001C0EAFF02C0EFFF07017B2907017D6F95
:1011600007017E6B8B909D9AAC80A0C07AF7A0C0DF
:10117000ADFFAC90010E07017B6F020E0701706F8F
:101180009D8807016F6B07016E6BE4CF0CF0E4CF15
:101190000BF0E4CF0AF0E4CF09F0E4CF08F0E4CF9D
:1011A00007F0E4CF06F0E4CF05F0E4CF04F0E4CF9D
:1011B00003F0E4CF02F0E4CF01F0E4CF00F012003E
:1011C000D9CFE5FFE1CFD9FF00C0E5FF01C0E5FFC2
:1011D00002C0E5FF03C0E5FF04C0E5FF05C0E5FF71
:1011E00006C0E5FF07C0E5FF08C0E5FF09C0E5FF51
:1011F0000AC0E5FF0BC0E5FF0CC0E5FF0DC0E5FF31
:101200000EC0E5FF0FC0E5FF10C0E5FF11C0E5FF10
:1012100012C0E5FF13C0E5FF14C0E5FF15C0E5FFF0
:1012200016C0E5FF17C0E5FF18C0E5FF19C0E5FFD0
:101230001AC0E5FF1BC0E5FF1CC0E5FF1DC0E5FFB0
:101240001EC0E5FF020EDBCF00F0030EDBCF01F086
:10125000040EDBCF02F0050EDBCF03F0060EDBCF72
:1012600004F0070EDBCF05F0080EDBCF06F0090E09
:10127000DBCF07F00A0EDBCF08F0096A0A6A02C06A
:101280000DF00D50800A0DE102500701566F01501C
:10129000556F0050546F070E016E540E006E800E95
:1012A000026E03C0E9FF04C0F3FF05501BEC26F0FB
:1012B0000B6E0B50D8B4CEEF0CF00B50250A02E0A9
:1012C000B5EF0CF00C6A0D6A0E6A0F6A106A0A0E0E
:1012D000116E126A136A146A200E156E1668176A68
:1012E0002B0E186E032A02E3044A052A03C0E9FF05
:1012F00004C0F3FF05501BEC26F0196E250A13E11C
:101300001950E56E0250E56E0150E56E0050E56E35
:101310007EEC1FF0040EE126094A0A2A032A02E3A2
:10132000044A052ABED71950300A06E1300E156E60
:10133000032A02E3044A052A03C0E9FF04C0F3FFBD
:1013400005501BEC26F02D0A06E1010E146E032A4F
:1013500002E3044A052A03C0E9FF04C0F3FF055075
:101360001BEC26F0200A08E1010E176E200E186E05
:10137000032A02E3044A052A03C0E9FF04C0F3FF7D
:1013800005501BEC26F02B0A06E1010E176E032A0E
:1013900002E3044A052A03C0E9FF04C0F3FF055035
:1013A0001BEC26F0196E800F4F0F2DE31950800FA4
:1013B000460F29E203C019F004C01AF005C01BF063
:1013C00019C0E9FF1AC0F3FF1B501BEC26F01C6E7E
:1013D000800F500F12E31C50800F460F0EE2135087
:1013E0000A0DF3CF1DF01D501C26D00E1C24136EC9
:1013F000192A02E31A4A1B2AE3D719C003F01AC0BC
:1014000004F01BC005F003C0E9FF04C0F3FF055062
:101410001BEC26F02E0A2EE1032A02E3044A052AD9
:10142000166A03C019F004C01AF005C01BF019C0F9
:10143000E9FF1AC0F3FF1B501BEC26F01C6E800F57
:10144000500F12E31C50800F460F0EE216500A0D8B
:10145000F3CF1DF01D501C26D00E1C24166E192A29
:1014600002E31A4A1B2AE3D719C003F01AC004F09A
:101470001BC005F003C0E9FF04C0F3FF05501BECDF
:1014800026F0196E6C0A07E1010E0C6E032A02E3C6
:10149000044A052A09D01950680A06E1010E0E6EA9
:1014A000032A02E3044A052A03C0E9FF04C0F3FF4C
:1014B00005501BEC26F0750A06E1010E106E032A9A
:1014C00002E3044A052A03C0E9FF04C0F3FF055004
:1014D0001BEC26F0196E730A05E1010E0D6E200E4D
:1014E000156E3FD01950780A03E1100E116E39D0F5
:1014F0001950580A05E1100E116E010E126E31D00E
:101500001950630A02E1116A2CD019506F0A03E1E5
:10151000080E116E26D01950660A03E1010E0F6EF7
:1015200020D01950640A1DE01950690A1AE01050C1
:1015300005E0FF0E03260422052213D01950E56EA4
:101540000250E56E0150E56E0050E56E7EEC1FF036
:10155000040EE126094A0A2A032A02E3044A052A5C
:10156000A0D60D5021E00650030F0D6E000E07208F
:10157000196E000E08201A6E0DC006F019C007F093
:101580001AC008F0FD0E0D26FF0E19221A220DC0FA
:10159000E9FF19C0F3FF1A5023EC25F00D6EF3CFCD
:1015A00019F0F4CF1AF032D10F50D8B43ED0065013
:1015B000040F0F6E000E07201B6E000E08201C6E1D
:1015C0000FC006F01BC007F01CC008F0FC0E0F2671
:1015D000FF0E1B221C220FC0E9FF1BC0F3FF1C5093
:1015E000E5EC24F00F6EF3CF1BF0F4CF1CF0E9CF45
:1015F0001DF0070E196E000E0D6E800E1A6E16503D
:10160000E56E240EE56E070EE56E000EE56E1D50CC
:10161000E56E1C50E56E1B50E56E0F50E56EA3ECB9
:1016200019F0080EE1261668F1D016680C5023E078
:101630000650040F0C6E000E07200F6E000E0820DF
:101640001B6E0CC006F00FC007F01BC008F0FC0EAC
:101650000C26FF0E0F221B220CC0E9FF0FC0F3FF68
:101660001B50E5EC24F00C6EF3CF0FF0F4CF1BF021
:10167000E9CF1CF06AD00E5032E00650020F0E6E19
:10168000000E07201D6E000E08201E6E0EC006F014
:101690001DC007F01EC008F0FE0E0E26FF0E1D2214
:1016A0001E220EC0E9FF1DC0F3FF1E50C9EC25F03D
:1016B0000E6E0EC00CF0E86A0EBEFF0E0F6E1B6EB3
:1016C0001C6E11500A0A03E11050D8B43ED00C50E1
:1016D0000E6E0EC00CF00F6A1B6A1C6A36D00650E4
:1016E000020F0E6E000E07201D6E000E08201E6EEB
:1016F0000EC006F01DC007F01EC008F0FE0E0E263C
:10170000FF0E1D221E220EC0E9FF1DC0F3FF1E505A
:10171000C9EC25F00E6EF3CF1DF00EC00CF01DC00D
:101720000FF0E86A1DBEFF0E1B6E1C6E11500A0AF8
:1017300002E110500AE00C500E6E0F501D6E0EC0EC
:101740000CF01DC00FF01B6A1C6A070E196E010E0B
:101750000D6E800E1A6E1150D8B440D0105013E0A8
:101760001150E56E070EE56E010EE56E1C50E56E3C
:101770001B50E56E0F50E56E0C50E56EB5EC1AF09F
:10178000070EE12612D01150E56E070EE56E010E30
:10179000E56E1C50E56E1B50E56E0F50E56E0C506B
:1017A000E56E78EC20F0070EE12617502FE00DC013
:1017B000E9FF19C0F3FF1A501BEC26F02D0A26E0B2
:1017C000FF0E0D2619221A2218C0E5FF0DC0E9FFF1
:1017D00019C0F3FF1A50BBEC26F018D00CC0E5FF7F
:1017E0000DC0E9FF19C0F3FF1A50BBEC26F00D50F5
:1017F000010F0C6E000E19200E6E000E1A20E56A05
:101800000CC0E9FF0EC0F3FFBBEC26F00DC00CF0DE
:1018100019C00EF01AC00FF013C010F0105010E0F5
:101820000CC0E9FF0EC0F3FF0F501BEC26F0176E43
:10183000175006E00C2A02E30E4A0F2A1006EED7D4
:1018400010C013F014501EE109C00CF00AC00EF0D5
:1018500010C00FF00F5010E01550E56E0250E56E0D
:101860000150E56E0050E56E7EEC1FF0040EE1269F
:101870000C4A0E2A0F06EED70CC009F00EC00AF073
:101880000FC013F016C00CF00DC00DF019C00EF013
:101890001AC00FF009C010F00AC015F00DC0E9FF22
:1018A0000EC0F3FF0F501BEC26F0166E1650D8B486
:1018B0003ED00CC016F0176A161E171E16501710D1
:1018C00005E00CC016F00C06165031E00DC0E9FF23
:1018D0000EC0F3FF0F501BEC26F0116E125010E0FB
:1018E0001150E56E86EC25F0166EE652165004E0B7
:1018F0001150166E169A02D011C016F016C011F0D3
:101900001150E56E0250E56E0150E56E0050E56E37
:101910007EEC1FF0040EE1260D2A02E30E4A0F2A88
:10192000104A152A1350D8B4B9D71306B7D710C028
:1019300009F015C00AF014502BE010C00CF015C0CF
:101940000DF013C00EF00E501FE0200EE56E025099
:10195000E56E0150E56E0050E56E7EEC1FF0040E62
:10196000E1260C4A0D2A0E06EED70B50E56E02500A
:10197000E56E0150E56E0050E56E7EEC1FF0040E42
:10198000E126094A0A2A04D00CC009F00DC00AF069
:10199000032A02E3044A052A51EF09F00AC0F3FFC3
:1019A0000950E4CF1EF0E4CF1DF0E4CF1CF0E4CFEB
:1019B0001BF0E4CF1AF0E4CF19F0E4CF18F0E4CF35
:1019C00017F0E4CF16F0E4CF15F0E4CF14F0E4CF35
:1019D00013F0E4CF12F0E4CF11F0E4CF10F0E4CF35
:1019E0000FF0E4CF0EF0E4CF0DF0E4CF0CF0E4CF35
:1019F0000BF0E4CF0AF0E4CF09F0E4CF08F0E4CF35
:101A000007F0E4CF06F0E4CF05F0E4CF04F0E4CF34
:101A100003F0E4CF02F0E4CF01F0E4CF00F0E4CF34
:101A2000D9FF120005C0E5FF06C0E5FF07C0E5FFCE
:101A300008C0E5FF09C0E5FF0AC0E5FF0BC0E5FFF0
:101A40000CC0E5FF0DC0E5FF0EC0E5FF0FC0E5FFD0
:101A500010C0E5FF11C0E5FF12C0E5FF13C0E5FFB0
:101A600014C0E5FF15C0E5FF16C0E5FF17C0E5FF90
:101A700018C0E5FF19C0E5FF1AC0E5FF1BC0E5FF70
:101A80001CC0E5FF1DC0E5FF000E00B0050F066A93
:101A9000F60F02E3062AFCD70A0F056E042E03D0C8
:101AA000FB0F01E3062A065000B0020F00B2050F3B
:101AB000076AF60F02E3072AFCD70A0F066E042E08
:101AC00003D0FB0F01E3072A075000B0060F00B256
:101AD000020F00B4050F086AF60F02E3082AFCD7CC
:101AE0000A0F076E042E03D0FB0F01E3082A0850EB
:101AF00000B2010F00B4020F00B6050F096AF60F1D
:101B000002E3092AFCD70A0F086E042E03D0FB0F4C
:101B100001E3092A095000B0090F00B2080F00B410
:101B2000060F00B6020F00B8050F0A6AF60F02E3AF
:101B30000A2AFCD70A0F096E042E03D0FB0F01E31B
:101B40000A2A0A5000B0030F00B2070F00B4050FB5
:101B500000B6010F00B8020F00BA050F0B6AF60FAE
:101B600002E30B2AFCD70A0F0A6E042E03D0FB0FE8
:101B700001E30B2A0B5000B0050F00B4010F00B6B3
:101B8000030F00B8060F00BA020F00BC050F0C6A65
:101B9000F60F02E30C2AFCD70A0F0B6E042E03D0BB
:101BA000FB0F01E30C2A0C5000B0070F00B2050F29
:101BB00000BA010F00BC020F00BE050F0D6AF60F40
:101BC00002E30D2AFCD70A0F0C6E042E03D0FB0F84
:101BD00001E30D2A0D5000B0070F00B2050F00B44D
:101BE000010F00B6020F00B8040F00BA080F00BCC6
:101BF000060F00BE020F01B0050F0E6AF60F02E3DA
:101C00000E2AFCD70A0F0D6E042E03D0FB0F01E342
:101C10000E2A0E5000B0040F00B2090F00B4090FD5
:101C200000B6080F00B8060F00BA020F00BC050F7F
:101C300000BE010F01B0020F01B2050F0F6AF60FCF
:101C400002E30F2AFCD70A0F0E6E042E03D0FB0FFF
:101C500001E30F2A0F5000B0040F00B2080F00B4C8
:101C6000070F00B6050F00B8010F00BA030F00BC44
:101C7000060F00BE030F01B0060F01B2020F01B440
:101C8000050F106AF60F02E3102AFCD70A0F0F6E39
:101C9000042E03D0FB0F01E3102A105000B0060FF2
:101CA00000B2020F00B4050F00B6010F00B8030F19
:101CB00000BA060F00BC020F00BE050F01B2010FF3
:101CC00001B4020F01B6050F116AF60F02E3112AE3
:101CD000FCD70A0F106E042E03D0FB0F01E3112A6C
:101CE000115000B0040F00B2090F00B4080F00B685
:101CF000070F00B8040F00BA080F00BC070F00BEA2
:101D0000040F01B0090F01B2080F01B4060F01B6AC
:101D1000020F01B8050F126AF60F02E3122AFCD770
:101D20000A0F116E042E03D0FB0F01E3122A12508A
:101D300000B4010F00B6030F00B8070F00BA040F7C
:101D400000BC090F00BE090F01B0080F01B2070F58
:101D500001B4050F01B6010F01B8020F01BA050F5A
:101D6000136AF60F02E3132AFCD70A0F126E042E31
:101D700003D0FB0F01E3132A135000B0060F00B28B
:101D8000020F00B4040F00B6080F00B8060F00BA27
:101D9000030F00BC060F00BE030F01B0070F01B216
:101DA000050F01B4010F01B6030F01B8060F01BA08
:101DB000020F01BC050F146AF60F02E3142AFCD7C8
:101DC0000A0F136E042E03D0FB0F01E3142A1450E4
:101DD00000B0090F00B2090F00B4080F00B6060FDB
:101DE00000B8030F00BA070F00BC040F00BE090FB4
:101DF00001B0080F01B2070F01B4050F01BA010FBE
:101E000001BC020F01BE050F156AF60F02E3152A89
:101E1000FCD70A0F146E042E03D0FB0F01E3152A22
:101E2000155000B0050F00B2010F00B4030F00B64B
:101E3000070F00B8050F00BC010F00BE020F01B074
:101E4000050F01B2010F01B4030F01B6070F01B86E
:101E5000040F01BA080F01BC060F01BE020F02B049
:101E6000050F166AF60F02E3162AFCD70A0F156E45
:101E7000042E03D0FB0F01E3162A165000B2010F07
:101E800000B4020F00B6040F00B8090F00BA090F22
:101E900000BC080F00BE060F01B0020F01B2050F13
:101EA00001B8010F01BA020F01BC050F01BE010FFD
:101EB00002B0020F02B2050F176AF60F02E3172AEB
:101EC000FCD70A0F166E042E03D0FB0F01E3172A6E
:101ED000175000BA010F00BC030F00BE070F01B07E
:101EE000050F01B4010F01B6020F01B8040F01BACA
:101EF000080F01BC060F01BE030F02B0060F02B2AD
:101F0000020F02B4050F186AF60F02E3182AFCD775
:101F10000A0F176E042E03D0FB0F01E3182A185086
:101F200001B0010F01B2030F01B4060F01B6020F99
:101F300001B8040F01BA080F01BC070F01BE050F5D
:101F400002B2010F02B4020F02B6050F196AF60FB2
:101F500002E3192AFCD70A0F186E042E03D0FB0FD8
:101F600001E3192A195001B6010F01B8020F01BA95
:101F7000040F01BC090F01BE090F02B0090F02B224
:101F8000080F02B4060F02B6020F02B8050F1A6A54
:101F9000F60F02E31A2AFCD70A0F196E042E03D09B
:101FA000FB0F01E31A2A1A5001BE010F02B0030F02
:101FB00002B2070F02B4050F02B6010F02B8020FFA
:101FC00002BA050F1B6AF60F02E31B2AFCD70A0FA1
:101FD0001A6E042E03D0FB0F01E31B2A1B5002B420
:101FE000010F02B6030F02B8060F02BA020F02BCBD
:101FF000050F1C6AF60F02E31C2AFCD70A0F1B6EA2
:10200000042E03D0FB0F01E31C2A1C5002BA010F5F
:1020100002BC020F02BE050F1D6AF60F02E31D2A65
:10202000FCD70A0F1C6E042E03D0FB0F01E31D2A00
:10203000300FEE6E1B50300FEE6E1A50300FEE6EFA
:102040001950300FEE6E1850300FEE6E1750300FE3
:10205000EE6E1650300FEE6E1550300FEE6E1450BF
:10206000300FEE6E1350300FEE6E1250300FEE6EDA
:102070001150300FEE6E1050300FEE6E0F50300FCB
:10208000EE6E0E50300FEE6E0D50300FEE6E0C50A7
:10209000300FEE6E0B50300FEE6E0A50300FEE6EBA
:1020A0000950300FEE6E0850300FEE6E0750300FB3
:1020B000EE6E0650300FEE6E0550300FEE6E170EBE
:1020C000E4CF1DF0E4CF1CF0E4CF1BF0E4CF1AF016
:1020D000E4CF19F0E4CF18F0E4CF17F0E4CF16F016
:1020E000E4CF15F0E4CF14F0E4CF13F0E4CF12F016
:1020F000E4CF11F0E4CF10F0E4CF0FF0E4CF0EF016
:10210000E4CF0DF0E4CF0CF0E4CF0BF0E4CF0AF015
:10211000E4CF09F0E4CF08F0E4CF07F0E4CF06F015
:10212000E4CF05F01200D9CFE5FFE1CFD9FF00C021
:10213000E5FF01C0E5FF02C0E5FF03C0E5FF04C005
:10214000E5FF05C0E5FF06C0E5FF07C0E5FF08C0E5
:10215000E5FF09C0E5FF0AC0E5FF0BC0E5FF0CC0C5
:10216000E5FF0DC0E5FF020ED924006E000EDA2057
:10217000016E800E026E030E0026000E0122022266
:10218000020EDBCF03F0030EDBCF04F0040EDBCF37
:1021900005F003C0E9FF04C0F3FF05501BEC26F077
:1021A000066E0EC0E5FF0FC0E5FF10C0E5FF03504F
:1021B000010F0E6E000E04200F6E000E0520106E33
:1021C000020E0EC0DBFF030E0FC0DBFF040E10C0BB
:1021D000DBFFE4CF10F0E4CF0FF0E4CF0EF006C049
:1021E00003F00650D8B448EF13F00350250A06E078
:1021F0000350E56E97EC26F0E652C2D7046A056AF2
:10220000020EDBCF06F0030EDBCF07F0040EDBCFB0
:1022100008F006C0E9FF07C0F3FF08501BEC26F0EA
:10222000036E0EC0E5FF0FC0E5FF10C0E5FF0650CE
:10223000010F0E6E000E07200F6E000E0820106EAC
:10224000020E0EC0DBFF030E0FC0DBFF040E10C03A
:10225000DBFFE4CF10F0E4CF0FF0E4CF0EF003503B
:10226000300A31E1020EDBCF06F0030EDBCF07F0C0
:10227000040EDBCF08F006C0E9FF07C0F3FF0850EB
:102280001BEC26F0036E0EC0E5FF0FC0E5FF10C08B
:10229000E5FF0650010F0E6E000E07200F6E000EB8
:1022A0000820106E020E0EC0DBFF030E0FC0DBFF16
:1022B000040E10C0DBFFE4CF10F0E4CF0FF0E4CF4A
:1022C0000EF0010E046E0350800F500FD8A069D09D
:1022D0000350800F460FD8B064D0056A020EDBCFE2
:1022E00006F0030EDBCF07F0040EDBCF08F003503F
:1022F000800F500F3BE30350800F460F37E2054439
:10230000E844FC0B096E055009260944FE0B0A6ED1
:1023100003500A24096ED00E0924056E06C0E9FF99
:1023200007C0F3FF08501BEC26F0036E062A02E3F9
:10233000074A082A0EC0E5FF0FC0E5FF10C0E5FF01
:1023400006C00EF007C00FF008C010F0020E0EC05D
:10235000DBFF030E0FC0DBFF040E10C0DBFFE4CF7A
:1023600010F0E4CF0FF0E4CF0EF0C1D70EC0E5FFC0
:102370000FC0E5FF10C0E5FF06C00EF007C00FF06C
:1023800008C010F0020E0EC0DBFF030E0FC0DBFF13
:10239000040E10C0DBFFE4CF10F0E4CF0FF0E4CF69
:1023A0000EF0070E07014C6F340E4B6F800E4D6F11
:1023B0004BC706F04CC707F04DC708F00701676B25
:1023C000035001E165D10350250A01E1FAD0096A01
:1023D0000350580A01E1092A0950D8A472D00350C9
:1023E000630A01E1ADD00A6A0350640A01E10A2AD6
:1023F0000A500CE10350730A01E1C2D00350750A80
:1024000005E00350780A01E15CD0E0D00050020FF3
:102410000B6E000E01200C6E000E02200D6E0BC024
:1024200000F00CC001F00DC002F0FE0E0B26FF0EF6
:102430000C220D220B500BC0E9FF0CC0F3FF0D5016
:10244000C9EC25F007015B6FF3CF5CF70A5014E08D
:102450005B510A6E5C510B6ED8800BAED8900CE3CA
:102460000B1C5C6F0A1C5B6F5B3F01D05C2B2D0E5D
:10247000E56EF7EC23F0E652270EE56E100EE56EE2
:102480005FEC23F0E652E652030EE56EE80EE56ED1
:102490005FEC23F0E652E652E56A640EE56E5FEC0F
:1024A00023F0E652E652E56A0A0EE56E5FEC23F091
:1024B000E652E65207015B51E56E93EC23F0E652DB
:1024C00085D009C066F70050020F096E000E01208A
:1024D0000A6E000E02200B6E09C000F00AC001F067
:1024E0000BC002F0FE0E0926FF0E0A220B2209C0C5
:1024F000E9FF0AC0F3FF0B50C9EC25F007015B6F41
:10250000F3CF5CF7100EE56E000EE56A5FEC23F08A
:10251000E652E652010EE56E000EE56A5FEC23F02E
:10252000E652E652E56A100EE56E5FEC23F0E652E5
:10253000E65207015B51E56E93EC23F0E65246D07C
:102540000050020F096E000E01200A6E000E0220DC
:102550000B6E09C000F00AC001F00BC002F0FE0EC5
:102560000926FF0E0A220B2209C0E9FF0AC0F3FF69
:102570000B50C9EC25F0E56EF7EC23F0E65226D0BF
:102580000050030F096E000E01200A6E000E02209B
:102590000B6E09C000F00AC001F00BC002F0FD0E86
:1025A0000926FF0E0A220B2209C0E9FF0AC0F3FF29
:1025B0000B5023EC25F0066EF3CF07F0F4CF08F0B4
:1025C00005D0250EE56EF7EC23F0E6524BC709F077
:1025D0004CC70AF04DC70BF0E56A09C0E9FF0AC015
:1025E000F3FF0B50BBEC26F006C04BF707C04CF7CF
:1025F00008C04DF74BC709F04CC70AF04DC70BF0A8
:1026000009C0E9FF0AC0F3FF0B501BEC26F0096E6E
:1026100007014B2B03E34C3F01D04D2B095006E043
:102620000550800F7F0F02E30506E4D705C009F0CF
:1026300005060950800F7F0F0DE3045003E0300EB4
:10264000096E02D0200E096E0950E56E97EC26F057
:10265000E652ECD706C004F007C005F008C006F04B
:1026600004C0E9FF05C0F3FF06501BEC26F0076E1F
:10267000042A02E3054A062A07C003F00750D8B42B
:10268000C0EF10F00350E56E97EC26F0E652E8D765
:10269000E4CF0DF0E4CF0CF0E4CF0BF0E4CF0AF080
:1026A000E4CF09F0E4CF08F0E4CF07F0E4CF06F080
:1026B000E4CF05F0E4CF04F0E4CF03F0E4CF02F080
:1026C000E4CF01F0E4CF00F0E4CFD9FF120000C066
:1026D000E5FF01C0E5FF02C0E5FF03C0E5FF04C060
:1026E000E5FF05C0E5FF06C0E5FF07C0E5FF070100
:1026F00079AB0BD0799B000EE56E390EE56E6C0E52
:10270000E56E1FEC23F0030EE126070179AD0BD037
:10271000799D000EE56E390EE56E760EE56E1FECC6
:1027200023F0030EE1260701715101E1CAD1010E28
:102730000701715DD8A0C3D1060E715DD8B0BFD1BD
:102740007105006EFA6AFB6A0034FA36E834FA362C
:10275000FC0B620FE56E270EFA22000EFB22E450FE
:10276000F96EBBEF13F032EF14F0A9EF14F0E6EFBF
:1027700014F023EF15F007017A39E8441F0B006EBF
:10278000016A240E0026070E012200C0E9FF01C0E5
:10279000EAFFEFCF02F0070E7A15036E010E046E0A
:1027A000056A035006E0E86CD89004360536010F40
:1027B000FCE302C006F0076A06500416075005162F
:1027C00004500510D8A47BD1010E046E035005E01F
:1027D000E86CD8900436010FFDE30450021200C0EB
:1027E000E9FF01C0EAFF02C0EFFF0A0EE56E97ECB9
:1027F00026F0E652730EE56E97EC26F0E652430E95
:10280000E56E97EC26F0E65207017A390F0B006E61
:102810000A0E005C05E20050016E300E012603D066
:10282000370E0024016E0150E56E97EC26F0E6525B
:102830000F0E07017A15006E0A0E005C05E20050CB
:10284000016E300E012603D0370E0024016E0150B8
:10285000E56E97EC26F0E6520A0EE56E97EC26F050
:10286000E6522DD107017A39E8441F0B006E016A48
:10287000240E0026070E012200C0E9FF01C0EAFF76
:10288000EFCF02F0070E7A15036E010E046E056A93
:10289000035006E0E86CD89004360536010FFCE3DF
:1028A00002C006F0076A06500416075005160450C9
:1028B0000510D8B404D1010E046E035005E0E86C95
:1028C000D8900436010FFDE3041C021600C0E9FF96
:1028D00001C0EAFF02C0EFFF0A0EE56E97EC26F09A
:1028E000E652730EE56E97EC26F0E652630EE56E47
:1028F00097EC26F0E65207017A390F0B006E0A0EAC
:10290000005C05E20050016E300E012603D0370E48
:102910000024016E0150E56E97EC26F0E6520F0E92
:1029200007017A15006E0A0E005C05E20050016E88
:10293000300E012603D0370E0024016E0150E56EE3
:1029400097EC26F0E6520A0EE56E97EC26F0E6527A
:10295000B6D00A0EE56E97EC26F0E652730EE56EE1
:1029600097EC26F0E652780EE56E97EC26F0E652EC
:1029700007017A390F0B006E0A0E005C05E2005069
:10298000016E300E012603D0370E0024016E015077
:10299000E56E97EC26F0E6520F0E07017A15006EF1
:1029A0000A0E005C05E20050016E300E012603D0D5
:1029B000370E0024016E0150E56E97EC26F0E652CA
:1029C0000A0EE56E97EC26F0E65279D00A0EE56E17
:1029D00097EC26F0E652730EE56E97EC26F0E65281
:1029E000610EE56E97EC26F0E65207017A390F0B7F
:1029F000006E0A0E005C05E20050016E300E0126EA
:102A000003D0370E0024016E0150E56E97EC26F0DE
:102A1000E6520F0E07017A15006E0A0E005C05E201
:102A20000050016E300E012603D0370E0024016ED7
:102A30000150E56E97EC26F0E6520A0EE56E97EC33
:102A400026F0E6523CD00A0EE56E97EC26F0E652F0
:102A5000730EE56E97EC26F0E652540EE56E97EC99
:102A600026F0E65207017A390F0B006E0A0E005C61
:102A700005E20050016E300E012603D0370E00240F
:102A8000016E0150E56E97EC26F0E6520F0E07013D
:102A90007A15006E0A0E005C05E20050016E300EE1
:102AA000012603D0370E0024016E0150E56E97EC2D
:102AB00026F0E6520A0EE56E97EC26F0E652070184
:102AC000716BE4CF07F0E4CF06F0E4CF05F0E4CF7C
:102AD00004F0E4CF03F0E4CF02F0E4CF01F0E4CF60
:102AE00000F0120000C0E5FF01C0E5FF02C0E5FFF5
:102AF00003C0E5FF6C50D8A440D13C0E0401001582
:102B0000006E0040E8403F0B0D0A01E0F6D00401E2
:102B10000451006E009E0050046F0051006E009E34
:102B20000050006F0701626B0701636B0701646B64
:102B300040C2E8FF41C200F000C042F70050050A61
:102B400009E1010E0701636F040E0701656F42C2C0
:102B50005FF78ED00050060A03E1C3EC1DF088D069
:102B60000050090A2EE1010E0701636F42C260F7AF
:102B70000701605104E1040E0701656F79D0050E6D
:102B80000701656F1E0E716E900E04010E6F020E2E
:102B90000F6F400E04010C6F1E0E726E200E0401AA
:102BA000116F200E126F020E136F880E0401106F4A
:102BB000000E0401166F020E176F400E0401146F11
:102BC00057D00050080A18E1010E0701636FF60E96
:102BD00007016025016E026A430E0222036A000E9D
:102BE0000322035007014A6F0250496F0150486F9A
:102BF000010E0701646F3CD0005003E107EC20F0A8
:102C000037D00050010A03E00050030A03E13BEC17
:102C100021F02ED000500A0A0EE1010E0701636F69
:102C2000000E07014A6F430E496FF40E486F010E04
:102C30000701646F1DD000500B0A06E00050200A07
:102C400003E00050220A04E1010E0701636F10D077
:102C50000050210A0DE1000E07014A6F440E496F32
:102C6000720E486F070E0701646F010E0701636F54
:102C7000070163510CE1100E0401016F400E026F59
:102C8000020E036F840E0401006F046F34D0020142
:102C900040AF1FD064C700F0016A0150475D02E1F8
:102CA0000050465D04E2020146510701646FDBEC0F
:102CB00020F0020E0701626F100E0401016F400E3A
:102CC000026F020E036F800E0401006FC80E046FC6
:102CD00012D0010E0701626F0401056BC80E0401DA
:102CE000046F100E0401016F800E026F020E036F5D
:102CF000C80E0401006F6D9862D007016251010A8D
:102D000001E038D00401015107016427800E07015A
:102D1000576F020E586F01C461F761C700F00701D9
:102D2000610700501DE059C700F05AC701F057C7AE
:102D300002F058C703F002C0E9FF03C0EAFFEFCF7B
:102D400002F00701573F01D0582B00C0E9FF01C036
:102D5000EAFF02C0EFFF0701593F01D05A2BDDD730
:102D6000040100AD03D0880E006F29D0C80E040105
:102D7000006F25D05CEC26F022D06C50040A1FE1D5
:102D80006E500BE107016551040A07E142C26EFF74
:102D90006E5003E1030E0701656F07016251020ADD
:102DA0000CE1DBEC20F0040104AD03D0880E046FCD
:102DB00006D0C80E0401046F02D05CEC26F0E4CF0C
:102DC00003F0E4CF02F0E4CF01F0E4CF00F0120012
:102DD00000C0E5FF01C0E5FF02C0E5FFABA202D0E5
:102DE0000701798BABA402D00701798D07017051DF
:102DF000010A36E19DBA0BD09EA208D0C6EC26F09F
:102E00009D921F0ECA6E6A0ECC6E9E923FD19EAAF4
:102E100026D0030ECA6E9D929E92AECF00F08B809C
:102E20009D9A9D98005018E007017E2B030E7E5D51
:102E300010E28B909D9AAC80A0C07AF7A0C0ADFF45
:102E4000AC90010E07017B6F020E0701706F9D8829
:102E50001DD1040E0701716F0701706B17D116D1D8
:102E600007017051030A01E066D09DBA0BD09EA203
:102E700008D0C6EC26F09D921F0ECA6E6A0ECC6E6C
:102E80009E9204D19EAA56D0AECF00F0B00E07019C
:102E90007225016E026A020E022201C0E9FF02C021
:102EA000EAFF00C0EFFF722B6A0ECC6E9E92725149
:102EB000010A1DE107017F6B3F0E00140701736FCC
:102EC000732B00500DE1030ECA6E9D929E928B8073
:102ED0009D9A9D980701706B010E0701716F07D0D5
:102EE00000AE03D00701798302D007017993005027
:102EF00007017F27070172510701735D1AE2030E74
:102F0000CA6E9D929E928B809D9A9D980701706BD0
:102F100007017F5109E10701720707017981010E5D
:102F20000701716FAD6A05D0030E0701716F010EC5
:102F3000AD6EACD0ABD007017051020A01E04DD0AC
:102F40009EA211D007017B5107017D190CE1030EF0
:102F5000CA6E9D929E920701706BC6EC26F08B8024
:102F60009D9A9D9893D09EB801D090D0030ECA6EC2
:102F70009D929E927BC701F007017B2B026AA00EF7
:102F80000126000E022201C0E9FF02C0EAFFEFCFD6
:102F9000ADFF7B5107017D191FE19D98070179A7BE
:102FA0000BD09D92070ECA6ED00ECC6E9E929D8263
:102FB000010E0701706F10D0070179A906D0C6EC89
:102FC00026F0050E0701706F07D09D92070ECA6E9E
:102FD000D00ECC6E9E929D8259D007017051040A8A
:102FE00029E1030ECA6E9D929E929EA84FD07BC788
:102FF00001F007017B2B026AA00E0126000E0222BF
:1030000001C0E9FF02C0EAFFEFCFADFF7B5107012E
:103010007D190FE19D989D92070ECA6ED00ECC6E61
:103020009E929D82050E0701706F0701736B070169
:10303000726B2CD007017051050A1FE19DBA09D0AF
:103040009EA206D0C6EC26F0030ECA6E9D929E92FA
:103050001DD09EAA11D0AECF00F0B00E0701722590
:10306000016E026A020E022201C0E9FF02C0EAFFFD
:1030700000C0EFFF722B0AD009D00701705106E1A2
:10308000030ECA6E9D929E929D989D9AE4CF02F087
:10309000E4CF01F0E4CF00F0120000C0E5FF01C072
:1030A000E5FF02C0E5FF03C0E5FF04C0E5FF05C082
:1030B000E5FF06C0E5FF07C0E5FF08C0E5FF09C062
:1030C000E5FF0AC0E5FF0BC0E5FF0CC0E5FF0DC042
:1030D000E5FF0EC0E5FF000E00B0010F00B2020FC9
:1030E00000B4040F00B6080F00B8060F00BA020FB4
:1030F00000BC040F00BE080F01B0060F01B2020FA2
:1031000001B4040F01B6080F01B8060F01BA020F8F
:1031100001BC040F01BE080F02B0060F02B2020F7D
:1031200002B4040F02B6080F02B8060F02BA020F6B
:1031300002BC040F02BE080F056AF60F02E3052A5F
:10314000FCD70A0F046E055000B8010F00BA030F38
:1031500000BC060F00BE020F01B0050F01B2010F47
:1031600001B4020F01B6040F01B8090F01BA090F2B
:1031700001BC080F01BE060F02B0030F02B2070F19
:1031800002B4040F02B6080F02B8070F02BA050F07
:10319000066AF60F02E3062AFCD70A0F056E0650F0
:1031A00000BE010F01B0020F01B2050F01BA010FFD
:1031B00001BC030F01BE070F02B0050F02B4010FDF
:1031C00002B6020F02B8050F02BA010F02BC030FCC
:1031D00002BE060F076AF60F02E3072AFCD70A0FA2
:1031E000066E075001B4010F01B6020F01B8040FBB
:1031F00001BA080F01BC060F01BE020F02B0050F95
:1032000002B2010F02B4020F02B6040F02B8080F97
:1032100002BA070F02BC040F02BE080F086AF60FBD
:1032200002E3082AFCD70A0F076E085001BC010F01
:1032300001BE030F02B0060F02B2030F02B4060F65
:1032400002B6020F02B8040F02BA090F02BC090F3E
:1032500002BE080F096AF60F02E3092AFCD70A0F1B
:10326000086E095002B2010F02B4020F02B6050F38
:1032700002BC010F02BE030F0A6AF60F02E30A2A1C
:10328000FCD70A0F096E0A5002B8010F02BA020FEA
:1032900002BC040F02BE080F0B6AF60F02E30B2AF2
:1032A000FCD70A0F0A6E0B500E6A0EE10A5010E1AD
:1032B000095012E1085014E1075016E1065018E1D8
:1032C00005501AE104501CD00E2A300FEE6E0A5041
:1032D0000E2A300FEE6E09500E2A300FEE6E085097
:1032E0000E2A300FEE6E07500E2A300FEE6E06508B
:1032F0000E2A300FEE6E05500E2A300FEE6E04507F
:103300000E2A300FEE6E0E50E4CF0EF0E4CF0DF02B
:10331000E4CF0CF0E4CF0BF0E4CF0AF0E4CF09F0F7
:10332000E4CF08F0E4CF07F0E4CF06F0E4CF05F0F7
:10333000E4CF04F0E4CF03F0E4CF02F0E4CF01F0F7
:10334000E4CF00F01200D9CFE5FFE1CFD9FF00C0F4
:10335000E5FF01C0E5FF02C0E5FF03C0E5FF04C0D3
:10336000E5FF05C0E5FF06C0E5FF07C0E5FF08C0B3
:10337000E5FF09C0E5FF0AC0E5FF0BC0E5FF020E4F
:10338000DBCF00F0030EDBCF01F0040EDBCF02F049
:10339000050EDBCF03F0060EDBCF04F0070EDBCF0C
:1033A00005F0080EDBCF06F0090EDBCF07F006C0F4
:1033B00008F0060608500EE006500424086EE86A7D
:1033C00006BEE8680520096E08C0E9FF09C0EAFFEB
:1033D000EF6AEDD700500701446F0150456F02506E
:1033E000466F0350476F44C700F045C701F046C71A
:1033F00002F047C703F0066A086A096A800E0314E0
:103400000A6E065007E1085005E1095003E10A5031
:10341000800A01E012D0039E00500701446F015062
:10342000456F0250466F0350476F04C0E9FF05C067
:10343000EAFF2D0EEF6E044A052A0701463547358F
:103440007E08006E4451016E4551026E7F0E461596
:10345000036E066A038E086A096A0A6A0B6A0050DC
:1034600019E0D88000AED8900EE30850082609363F
:103470000A360B3603BE0880015001260236033699
:103480000636002AECD7D8900632033202320132D7
:103490000006E5D7085009100A100B1012E005507D
:1034A000E56E0450E56E0B50E56E0A50E56E09506E
:1034B000E56E0850E56E26EC24F0006E060EE1265F
:1034C00008D004C0E9FF05C0EAFF300EEF6E010E20
:1034D000006E00500426E86A00BEE8680522075026
:1034E00028E004C0E9FF05C0EAFF2E0EEF6E002AB7
:1034F000044A052A07501808E56E0550E56E045089
:10350000E56E0650E56E0350E56E0250E56E015023
:10351000E56EC5EC23F0016E070EE1260150002692
:1035200007500426E86A052204C0E9FF05C0EAFF47
:10353000EF6A0050E4CF0BF0E4CF0AF0E4CF09F0DB
:10354000E4CF08F0E4CF07F0E4CF06F0E4CF05F0D5
:10355000E4CF04F0E4CF03F0E4CF02F0E4CF01F0D5
:10356000E4CF00F0E4CFD9FF1200D9CFE5FFE1CFDF
:10357000D9FF00C0E5FF01C0E5FF02C0E5FF03C0C1
:10358000E5FF04C0E5FF05C0E5FF06C0E5FF07C095
:10359000E5FF08C0E5FF09C0E5FF0AC0E5FF0BC075
:1035A000E5FF0CC0E5FF0DC0E5FF0EC0E5FF0FC055
:1035B000E5FF020EDBCF00F0030EDBCF01F0040EBF
:1035C000DBCF02F0050EDBCF03F0060EDBCF04F0FD
:1035D000070EDBCF05F0080EDBCF06F0200E076EDE
:1035E000086A06C009F00A6A0B6A0C6AE56AE56AAD
:1035F000E56A0950E56E0350E56E0250E56E015034
:10360000E56E0050E56E5FEC1EF00D6E080EE126D3
:10361000300E0D263A0E0D5C05E30D500E6E270E92
:103620000E240D6EFF0E07260822E00E07240E6EF4
:10363000000E08200F6E0EC0E9FF0FC0EAFF0DC09C
:10364000EFFF0C50E56E0B50E56E0A50E56E095029
:10365000E56E0350E56E0250E56E0150E56E0050D8
:10366000E56EF2EC1EF0006EF3CF01F0F4CF02F045
:10367000E9CF03F0080EE1260050011002100310FC
:10368000D8A4AFD707C000F008C001F004C002F012
:1036900005C003F000C004F001C005F0004A012A93
:1036A000E00E0426000E052204C0E9FF05C0EAFF73
:1036B000EFCF04F002C0E9FF03C0EAFF04C0EFFF50
:1036C000024A032A000E015C02E1200E005CE2E3E4
:1036D00002C0E9FF03C0EAFF000EEF6AE4CF0FF07B
:1036E000E4CF0EF0E4CF0DF0E4CF0CF0E4CF0BF01C
:1036F000E4CF0AF0E4CF09F0E4CF08F0E4CF07F01C
:10370000E4CF06F0E4CF05F0E4CF04F0E4CF03F01B
:10371000E4CF02F0E4CF01F0E4CF00F0E4CFD9FF32
:10372000120000C0E5FF01C0E5FF67EC13F00701E0
:103730007051050A28E107017251070173191CE055
:10374000070172510701731915E073C700F00701F3
:10375000732B016AB00E0026020E012200C0E9FFA1
:1037600001C0EAFFEFCF00F00050E56E97EC26F0C5
:10377000E652E6D7D7EC26F007016E51D8B4A1D0B7
:1037800015EC04F09ED0F29E07017051D8A45CD0D5
:10379000030ECA6E9D929E9207016E5103E015ECD6
:1037A00004F08FD0070179B18CD007017451070163
:1037B000805DD8A086D0806B0701772B77510701F9
:1037C000765D07E2010E0701776F020E0701786F41
:1037D00003D007017835783707017739E8441F0BA4
:1037E000006E016AF00E0026020E012200C0E9FF01
:1037F00001C0EAFFEFCF00F007017851001600503A
:10380000D8B45FD00701736B0701726B07017F6B40
:10381000AC808B909D9A67EC13F0F29C77C77AF797
:10382000800E07017711AD6EAC90800E7711AD6EF2
:103830009D92070ECA6ED00ECC6E9E929D82030E94
:103840000701706FF28C3DD007017051010A25E12C
:103850009DAA37D09EA235D0030ECA6E9D929E922D
:103860008B809D9A9D9807017E2B7E5D10E28B9048
:103870009D9AAC80A0C07AF7A0C0ADFFAC90010EBD
:1038800007017B6F020E0701706F9D881AD0050E2D
:103890000701716F0701706B14D007017051030AA3
:1038A00010E19DAA0ED09EA20CD0030ECA6E9D926E
:1038B0009E92020E0701716F8B809D9A9D98070161
:1038C000706BF28E1FEC1DF0E4CF01F0E4CF00F03E
:1038D0001200D9CFE5FFE1CFD9FF00C0E5FF01C05D
:1038E000E5FF02C0E5FF020EDBCF00F0030EDBCFE9
:1038F000A8FF00C0A9FFA69EA69CA684F29E550E16
:10390000A76EAA0EA76EA682A6A202D00000FCD7C0
:10391000A6A610D0000E026E390E016E4A0E006E81
:103920000250E56E0150E56E0050E56E1FEC23F08D
:10393000030EE126A694F28EE4CF02F0E4CF01F06C
:10394000E4CF00F0E4CFD9FF12004552524F523A73
:103950002077726974696E6720746F2045455052F4
:103960004F4D206661696C6564210A004F455252D3
:103970002021210A0000464552522021210A000040
:10398000732066726169736520696E69742E2E2ECC
:103990000A000A7320667261697365206C6F672084
:1039A0003A0A000046726169736553746174652058
:1039B0003A202564203B2046726169736553746127
:1039C0007475733A2025640A000025643A25642042
:1039D00000005175697420626F6F746C6F6164656B
:1039E00072206D6F64652E0A000073562055736255
:1039F00046726169736520322E312E34202844507E
:103A00005F5553422F534443432920412E526F7533
:103A1000737365617520323031330A007349442570
:103A20006325630A0000456E74657220626F6F74CF
:103A30006C6F61646572206D6F64652E0A0000C052
:103A4000E5FF01C0E5FF02C0E5FF03C0E5FF070198
:103A500079A190D0070177390F0B006E070179B378
:103A600000860050016E300E0124006E3A0E005C9C
:103A700005E30050016E070E0124006E0050E56E54
:103A800097EC26F0E6520F0E07017715016E300E07
:103A90000124006E3A0E005C05E30050016E070E33
:103AA0000124006E0050E56E97EC26F0E652070107
:103AB00079A31BD0010E016E07017251015CD8B0D1
:103AC0004ED001C002F0012A036AB00E0226020E97
:103AD000032202C0E9FF03C0EAFFEFCF02F0025069
:103AE000E56E97EC26F0E652E7D7010E016E07016E
:103AF0007251015C34E201C002F0012A036AB00E87
:103B00000226020E032202C0E9FF03C0EAFFEFCF44
:103B100002F002380F0B036E300E0324006E3A0ED3
:103B2000005C05E30050036E070E0324006E005096
:103B3000E56E97EC26F0E6520F0E0216300E0224C8
:103B4000006E3A0E005C05E30050026E070E022480
:103B5000006E0050E56E97EC26F0E652C8D70A0ECC
:103B6000E56E97EC26F0E6520701726B0701736B66
:103B700007017991E4CF03F0E4CF02F0E4CF01F044
:103B8000E4CF00F0120000C0E5FF01C0E5FF02C075
:103B9000E5FF03C0E5FF04C0E5FF02014051800AD4
:103BA00001E082D043C200F042C201F00050010A9D
:103BB0001AE1010E0701636FD80E0701486F430E2B
:103BC000496F000E4A6F48C702F049C703F04AC761
:103BD00004F002C0F6FF03C0F7FF04C0F8FF0900BD
:103BE000F5CF64F761D00050060A0EE1010E07011F
:103BF000636FEA0E0701486F430E496F000E4A6F6C
:103C00000A0E0701646F50D00050020A1CE1010E39
:103C10000701636F000E07014A6F430E496FFC0EE8
:103C2000486F020F026E000E4921036E000E4A21FA
:103C3000046E02C0F6FF03C0F7FF04C0F8FF0900DE
:103C4000F5CF64F731D00050030A2EE1010E0701D1
:103C5000636F015008E1400E0701486F440E496F41
:103C6000000E4A6F12D00150010A08E1440E07010C
:103C7000486F440E496F000E4A6F07D0520E07017D
:103C8000486F440E496F000E4A6F48C700F049C79D
:103C900001F04AC702F000C0F6FF01C0F7FF02C002
:103CA000F8FF0900F5CF64F7E4CF04F0E4CF03F0A8
:103CB000E4CF02F0E4CF01F0E4CF00F01200D9CF5E
:103CC000E5FFE1CFD9FF00C0E5FF01C0E5FF02C07D
:103CD000E5FF03C0E5FF04C0E5FF05C0E5FF06C042
:103CE000E5FF07C0E5FF08C0E5FF09C0E5FF0AC022
:103CF000E5FF020EDBCF00F0030EDBCF01F0040E78
:103D0000DBCF02F0050EDBCF03F0060EDBCF04F0B5
:103D1000070EDBCF05F0080EDBCF06F0090EDBCF78
:103D200007F0086A096A0750800BE8440A6E0A50D7
:103D30001BE1045004260536063607360750035C9F
:103D400008E10650025C05E10550015C02E1045007
:103D5000005C06E2D890073206320532043204D005
:103D6000092A09C008F0DFD70750035C08E10650B4
:103D7000025C05E10550015C02E10450005C08E3CF
:103D80000450005E0550015A0650025A0750035A6B
:103D9000D890073206320532043208C009F008060E
:103DA0000950E2E103C0E9FF02C0F4FF01C0F3FFE4
:103DB0000050E4CF0AF0E4CF09F0E4CF08F0E4CFFC
:103DC00007F0E4CF06F0E4CF05F0E4CF04F0E4CF51
:103DD00003F0E4CF02F0E4CF01F0E4CF00F0E4CF51
:103DE000D9FF1200D9CFE5FFE1CFD9FF00C0E5FF31
:103DF00001C0E5FF02C0E5FF03C0E5FF04C0E5FF29
:103E000005C0E5FF06C0E5FF07C0E5FF08C0E5FF08
:103E100009C0E5FF0AC0E5FF0BC0E5FF0CC0E5FFE8
:103E20000DC0E5FF020EDBCF00F0030EDBCF01F08B
:103E3000040EDBCF02F0050EDBCF03F0060EDBCF66
:103E400004F0070EDBCF05F0080EDBCF06F0090EFD
:103E5000DBCF07F0086A096A0A6A0B6A200E0C6E4B
:103E60000350800BE8440D6E0050002601360236E8
:103E700003360850082609360A360B360D50D8A4EA
:103E8000088007500B5C08E106500A5C05E105500C
:103E9000095C02E10450085C09E30450085E055027
:103EA000095A06500A5A07500B5A00800C2ED8D7D0
:103EB00003C0E9FF02C0F4FF01C0F3FF0050E4CFEC
:103EC0000DF0E4CF0CF0E4CF0BF0E4CF0AF0E4CF38
:103ED00009F0E4CF08F0E4CF07F0E4CF06F0E4CF38
:103EE00005F0E4CF04F0E4CF03F0E4CF02F0E4CF38
:103EF00001F0E4CF00F0E4CFD9FF1200D9CFE5FF05
:103F0000E1CFD9FF00C0E5FF01C0E5FF02C0E5FF3A
:103F100003C0E5FF04C0E5FF05C0E5FF06C0E5FFFF
:103F200007C0E5FF020EDBCF00F0030EDBCF01F090
:103F3000040EDBCF02F0050EDBCF03F002C006F06B
:103F40000650046E800A33E100C0E9FF01C0F3FFB0
:103F5000025023EC25F0056EF3CF06F0F4CF07F006
:103F600003C0E5FF05C0E9FF06C0F3FF0750BBEC47
:103F700026F000C0E9FF01C0F3FF025023EC25F05A
:103F8000056EF3CF06F0F4CF07F0052A02E3064AE8
:103F9000072A05C0E5FF06C0F4FF07C0F6FF00C012
:103FA000E9FF01C0F3FF02507AEC26F01DD004AA0D
:103FB0001BD0047A045004E10350E5EC26F014D041
:103FC0000450010A04E10350F1EC26F00DD0045036
:103FD0000F0A04E1035097EC26F006D004500E0AB5
:103FE00003E10350ECEC26F0E4CF07F0E4CF06F059
:103FF000E4CF05F0E4CF04F0E4CF03F0E4CF02F027
:10400000E4CF01F0E4CF00F0E4CFD9FF120000C00C
:10401000E5FF01C0E5FF02C0E5FF03C0E5FF04C006
:10402000E5FF1F0E02014015006E00500BE1010E6E
:104030000701636F000E07014A6F430E496FFA0EC6
:10404000486F45D00050010A0BE1000E07014A6F8E
:10405000430E496FF40E486F010E0701636F37D0AE
:104060000050020A34E10F0E02014415006E800E6A
:104070004415016E010E0701636F000E026E040EFF
:10408000036E0050080DF450046EF3CF00F00050A2
:1040900002240701596F045003205A6F015004E0B5
:1040A000040E592701E35A2B59C700F05AC701F0F3
:1040B00000C0E9FF01C0EAFFEFCF00F000A407D085
:1040C000000E07014A6F430E496FF80E486F070153
:1040D000635103E0020E0701646FE4CF04F0E4CF04
:1040E00003F0E4CF02F0E4CF01F0E4CF00F01200DF
:1040F000D9CFE5FFE1CFD9FF00C0E5FF01C0E5FF63
:1041000002C0E5FF03C0E5FF04C0E5FF05C0E5FF11
:1041100006C0E5FF020EDBCF00F0030EDBCF01F09F
:10412000040EDBCF02F0050EDBCF03F0060EDBCF73
:1041300004F0070EDBCF05F0080EDBCF06F0D880C9
:1041400003AED89015E306500A0A12E104C0E9FF55
:1041500005C0EAFF2D0EEF6E044A052A031E021E5B
:10416000011E006C05E1012A03E1022AD8B4032AEA
:104170000650E56E0550E56E0450E56E0350E56EA1
:104180000250E56E0150E56E0050E56EB5EC1AF098
:10419000070EE126E4CF06F0E4CF05F0E4CF04F00B
:1041A000E4CF03F0E4CF02F0E4CF01F0E4CF00F07D
:1041B000E4CFD9FF120000C0E5FF01C0E5FF02C057
:1041C000E5FF03C0E5FF04C0E5FF100E0701645DD5
:1041D00003E264C700F002D0100E006E0401045127
:1041E000016EFC0E01160150046F00500401056FB2
:1041F000800E066F020E076F00500701645F800E8D
:104200000701596F020E5A6F00C061F761C700F0D5
:1042100007016107005024E059C700F05AC701F0B8
:1042200048C702F049C703F04AC704F002C0F6FFCE
:1042300003C0F7FF04C0F8FF0900F5CF02F0070143
:10424000482B03E3493F01D04A2B00C0E9FF01C0DE
:10425000EAFF02C0EFFF0701593F01D05A2BD6D722
:10426000E4CF04F0E4CF03F0E4CF02F0E4CF01F0B8
:10427000E4CF00F0120000C0E5FF01C0E5FF02C07E
:10428000E5FF03C0E5FF04C0E5FF1F0E0201401576
:1042900042C201F0020A01E03DD00F0E02014415B6
:1042A000006E800E4415026E015034E1005032E081
:1042B000010E0701636F000E016E040E036E0050C5
:1042C000080DF450046EF3CF00F0005001240701F4
:1042D000596F045003205A6F025004E0040E59270E
:1042E00001E35A2B02014151030A03E1840E006EDF
:1042F00007D00250010A02E1006A02D0880E006E67
:1043000059C701F05AC702F001C0E9FF02C0EAFF35
:1043100000C0EFFFE4CF04F0E4CF03F0E4CF02F0FD
:10432000E4CF01F0E4CF00F0120000C0E5FF01C0CF
:10433000E5FF07016E6B07016F6B0701796B0701E2
:10434000706B0701716B0701726B0701736B0701DB
:10435000746B080EB86EE56A2F0EE56E3E0EDBEC50
:1043600022F0E652E65207018183CA6ACA82CA80F5
:10437000CB68CA848B909D9A0701756BF00E07017C
:104380007525006E016A020E012200C0E9FF01C01E
:10439000EAFFEF6A240E7525006E016A070E0122FE
:1043A00000C0E9FF01C0EAFFEF6A752B100E755DD2
:1043B000E5E3040E0701766F010E0701776F020E29
:1043C0000701786F9D929F829F889F8AF28EE4CF2B
:1043D00001F0E4CF00F01200120100020200001010
:1043E00008040A000001010000010A0600020200A0
:1043F000001001000000000101000100090243005B
:10440000020100C03209040000010202010005247B
:104410000010010524010101042402020524060004
:10442000010705810308000A09040100020A0000CF
:10443000020705020220000007058202200000009A
:10444000040309040E03540065007300740069003E
:104450002100200355005300420020004700650062
:104460006E00650072006900630020004300440094
:104470004300802500000000080000C0E5FF006A3E
:104480006FBE002A0050010A09E00701655106E0ED
:10449000006A6DB2002A0050010A01E13BD068A019
:1044A0001CD069A01AD06A6A686A9F0E6B6E2B0EC8
:1044B000696E6E6A160E706E006A68B6002A005049
:1044C000010A02E16896F8D76D985CEC26F00701C6
:1044D000606B030E0701656F689068AC02D069BC21
:1044E000689C68AA0CD069AA0AD0006A70B0002A39
:1044F0000050010A03E15CEC26F07090689A68A213
:1045000002D069B2689268A605D069A603D072ECA1
:1045100015F06896E4CF00F01200BC0EF66E4D0E5A
:10452000F76E000EF86E0900F550056E0900F550A3
:10453000066E04E1056702D0DAEF22F00900F550BB
:10454000006E0900F550016E0900F550026E090079
:104550000900F550E96E0900F550EA6E09000900FE
:104560000900F550036E0900F550046E09000900BA
:10457000F6CF07F0F7CF08F0F8CF09F000C0F6FF4C
:1045800001C0F7FF02C0F8FF035002E1045007E04A
:104590000900F550EE6E0306F8E20406F9D707C0ED
:1045A000F6FF08C0F7FF09C0F8FF050601E206069E
:1045B00099EF22F01200D9CFE5FFE1CFD9FF00C07B
:1045C000E5FF01C0E5FF02C0E5FF006E020EDBCF94
:1045D00001F0030EDBCF02F0AC6AAB6A00B0AC882E
:1045E00000A202D0AC8CAB8C00A401D0AC8E00A693
:1045F00002D0AB8801D0AB8A00A803D0AC84B886C7
:1046000001D0B8969E9800AC02D09D8A01D09D9AA8
:104610009E9A00AE02D09D8801D09D980250B06E47
:104620000150AF6E948C948EAC8AAB8EE4CF02F0C6
:10463000E4CF01F0E4CF00F0E4CFD9FF1200D9CFEE
:10464000E5FFE1CFD9FF00C0E5FF01C0E5FF02C0F3
:10465000E5FF020ED924006E000EDA20016E800EF6
:10466000026E030E0026000E012202220250E56EA9
:104670000150E56E0050E56E040EDBCFE5FF030E42
:10468000DBCFE5FF020EDBCFE5FF07015051E56E02
:104690004F51E56E4E51E56EE0EC08F0006EF3CF41
:1046A00001F0090EE12601C0F3FF0050E4CF02F053
:1046B000E4CF01F0E4CF00F0E4CFD9FF1200D9CF6E
:1046C000E5FFE1CFD9FF00C0E5FF01C0E5FF02C073
:1046D000E5FF020EDBCF00F0030EDBCF01F0026A34
:1046E000015007015C5D02E100505B5D07E3005093
:1046F00007015B5F01505C5B022AF2D702C000F049
:104700000701675102E1025005E00050E56E93ECAD
:1047100023F0E652E4CF02F0E4CF01F0E4CF00F062
:10472000E4CFD9FF1200D9CFE5FFE1CFD9FF00C018
:10473000E5FF01C0E5FF02C0E5FF020EDBCF00F0A0
:104740000050800F760F03E2300E016E0BD0070190
:10475000665103E0410E026E02D0610E026EF60E4B
:104760000224016E015000260050E56EF7EC23F0A4
:10477000E652010E0701676FE4CF02F0E4CF01F0CB
:10478000E4CF00F0E4CFD9FF1200D9CFE5FFE1CFAD
:10479000D9FF00C0E5FF01C0E5FF02C0E5FF03C08F
:1047A000E5FF04C0E5FF020EDBCF00F0030EDBCF18
:1047B00001F0040EDBCF02F0050EDBCF03F0060E96
:1047C000DBCFE9FF070EDBCFEAFF080EDBCF04F0FB
:1047D00012EC0DF0E4CF04F0E4CF03F0E4CF02F0EC
:1047E000E4CF01F0E4CF00F0E4CFD9FF1200D9CF3D
:1047F000E5FFE1CFD9FF00C0E5FF01C0E5FF02C042
:10480000E5FF03C0E5FF020EDBCF00F04BC701F070
:104810004CC702F04DC703F000C0E5FF01C0E9FF3F
:1048200002C0F3FF0350BBEC26F007014B2B03E360
:104830004C3F01D04D2BE4CF03F0E4CF02F0E4CFA6
:1048400001F0E4CF00F0E4CFD9FF1200D9CFE5FFAB
:10485000E1CFD9FF00C0E5FF01C0E5FF02C0E5FFE1
:1048600003C0E5FF020EDBCF00F0030EDBCF01F04B
:10487000040EDBCF02F0050EDBCF03F0060EDBCF1C
:10488000E9FF070EDBCFEAFF4DEC18F0E4CF03F0B1
:10489000E4CF02F0E4CF01F0E4CF00F0E4CFD9FFA1
:1048A000120000C0E5FF01C0E5FF02C0E5FF006E99
:1048B000B3EC25F0016E0150FBE140C701F00701A8
:1048C000402B026A000E0126020E022201C0E9FFFF
:1048D00002C0EAFF00C0EFFF200E405DD8B0D7EC69
:1048E00026F0E4CF02F0E4CF01F0E4CF00F01200B4
:1048F00000C0E5FF01C0E5FF2CEC26F0006E005083
:10490000FBE041C700F00701412B016A200E0026A1
:10491000020E012200C0E9FF01C0EAFFEFCF00F064
:10492000040111510701415DD8B06BEC26F0005035
:10493000E4CF01F0E4CF00F0120000C0E5FF6DC746
:1049400000F007016D2B0050C80A13E107016D6BE1
:10495000006A8BB2002A0050D880E866D890006ABE
:1049600000360050010BE844F46E8B50FD0BF41040
:104970008B6E0701802B805102E1FF0E8069E4CF2E
:1049800000F01200D8CFE5FFE0CFE5FFE56EF3CFF2
:10499000E5FFF4CFE5FFE9CFE5FFEACFE5FFFACF8A
:1049A000E5FFFBCFE5FFE4CFFBFFE4CFFAFFE4CF69
:1049B000EAFFE4CFE9FFE4CFF4FFE4CFF3FFE450F4
:1049C000E4CFE0FFE4CFD8FF1000E8AE0AD0F3CF89
:1049D000EAFFEE50EECFF3FFEECFF4FFEECFE9FFAC
:1049E0001200E8BCFDEF26F0E9CFF6FFF3CFF7FFAA
:1049F000F86E0900F5500900F5CFF3FF0900F5CF77
:104A0000F4FF0900F5CFE9FF1200F3CFE5FFF4CF83
:104A1000E5FFE9CFE5FFEACFE5FFFACFE5FFFBCF02
:104A2000E5FFA1AA03D03DEC22F0A19AE4CFFBFF61
:104A3000E4CFFAFFE4CFEAFFE4CFE9FFE4CFF4FFED
:104A4000E4CFF3FF1100E8AE08D0F3CFEAFFEE5059
:104A5000EECFF3FFEECFF4FF1200E8BCF7EF26F045
:104A6000E9CFF6FFF3CFF7FFF86E0900F550090024
:104A7000F5CFF3FF0900F5CFF4FF120007014E6BED
:104A80004F6B2F0E506F9DEC25F0B0EC26F08B9203
:104A9000F28CF28E07016551050A02E08B82FAD78B
:104AA000E9EC26F097EC26F0FBD71200F2CFEAFFF4
:104AB000F29EA69EA69CA684E9CFA9FFE4CFA8FFFC
:104AC000CFEC26F0F4CFA8FFCFEC26F0F6CFA8FF6E
:104AD000CFEC26F0A694EABEF28E1200F2CFF6FFDB
:104AE000F29EA69EA69CE9CFA9FFA680A850A92A5F
:104AF000A680A8CFF3FFA92AA680A8CFF4FFA92AF1
:104B0000A680A8CFEAFFF6BEF28E1200D9CFE5FF4D
:104B1000E1CFD9FF00C0E5FF020EDBCF00F0610E50
:104B2000005C05E37B0E005C02E2010E01D0E86A46
:104B3000E4CF00F0E4CFD9FF1200140E6F6E07012E
:104B4000656B0701606B6DB606D06D6A696A6D862C
:104B5000010E0701656F686A696A6980020E0701C4
:104B6000656FA08A120000C0E5FF800E04011415D5
:104B7000006E005003E1006A002A01D0006A005074
:104B8000D880E866D890006A00360050E4CF00F084
:104B90001200E8AE06D0F3CFEAFFEE50EECFF3FFFF
:104BA0001200E8BCF5EF26F0E9CFF6FFF3CFF7FFF0
:104BB000F86E0900F5500900F5CFF3FF120000C0B0
:104BC000E5FF006E00500CE000500401156F040179
:104BD00014AD03D0880E146F03D0C80E0401146FF7
:104BE000E4CF00F0120011EEFFF021EEFFF0F86AC2
:104BF000A68EA69CE9680E0EEA6E0068000EED6AAD
:104C00000050FDE18DEC22F03EEC25F0FFD7F2CF15
:104C1000F6FFF29EA69EA69CE9CFA9FFA680A8500B
:104C2000A92AA680A8CFF3FFA92AA680A8CFF4FFBF
:104C3000F6BEF28E1200E8AE04D0F3CFEAFFEE50DB
:104C40001200E8BCF9EF26F0E9CFF6FFF3CFF7FF4B
:104C5000F86E0900F5501200040110AF02D0E86AA6
:104C60000AD0040111510701415D04E36BEC26F009
:104C7000E86A01D0010E1200F2CFF6FFF29EA69E66
:104C8000A69CE9CFA9FFA680A850A92AA680A8CFF4
:104C9000F3FFF6BEF28E1200F2CFEAFFF29EA69E5E
:104CA000A69CA684E9CFA9FFE4CFA8FFCFEC26F00D
:104CB000A694EABEF28E12000701626B100E040188
:104CC000016F400E026F020E036F880E0401006F29
:104CD000046B6D9812000701416B200E0401116FE7
:104CE000040110AD03D0880E106F03D0C80E04016C
:104CF000106F1200E8AE09D0F3CFEAFFE4CFEEFF69
:104D0000F4CFEEFFF6CFEEFF1200E8BCFBEF26F08B
:104D10001200D9CFE5FFE1CFD9FF020EDBCFA9FF0B
:104D2000A69CA69EA680A850E4CFD9FF120000C082
:104D3000E5FF006E51EC24F000500A0A02E1D7ECC6
:104D400026F0E4CF00F01200F2CFF6FFF29EA69E0E
:104D5000A69CE9CFA9FFA680A850F6BEF28E12004D
:104D60000F0EC112B56A8B6A9468FC0E8B169416EE
:104D7000948494901200E8AE05D0F3CFEAFFE4CF1C
:104D8000EEFF1200E8BCF3EF26F01200ACA2FED753
:104D9000AE50AB98AB889D8A9D988B801200550EC3
:104DA000A76EAA0EA76EA682A6B2FED7A94A0701D1
:104DB0004051DFEC25F00701406B12000100DE4D91
:104DC00000004007000004000000ACA2FED7AD6E5A
:104DD000120078EC24F01200E8CF7FFF12000000F0
:104DE0000000C96E12004CEF26F03CEF26F007EFF2
:0E4DF00026F0A4EF26F056EF25F06EEF25F02A
:00000001FF
